:020000040800F2
:1000000050050020D9000008A9170008B9150008FC
:1000100000000000000000000000000000000000E0
:10002000000000000000000000000000551800085B
:100030000000000000000000F11700085718000839
:10004000EB000008EB000008EB000008EB000008E4
:10005000F3170008EB000008EB000008EB000008B5
:1000600000000000EB000008EB000008EB000008B7
:10007000EB000008EB00000800000000EB000008A7
:1000800000000000EB00000800000000000000007D
:10009000EB00000800000000EB000008EB00000887
:1000A000EB000008EB000008EB0000086D1D0008E5
:1000B000EB000008EB00000800000000000000005A
:1000C0000448854600F090F800480047411F0008AA
:1000D000C046C046500500200448804704480047F9
:1000E000FEE7FEE7FEE7FEE7FEE7FEE7D5180008BD
:1000F000C100000830B50B46014600202022012433
:1001000009E00D46D5409D4205D31D469540491B4B
:100110002546954040191546521E002DF1DC30BD94
:10012000F0B51FB40646002082B005464024019178
:1001300000901BE0019922460F46304600F042F83D
:10014000049A059B801A994110D3104619462246FD
:1001500000F028F8361A8F4101972246012000212D
:10016000009F00F01FF838184D4100902046641E93
:100170000028DFDC019B00982946324607B0F0BD1D
:10018000D2B201E00270401C491EFBD2704700222F
:10019000F6E710B513460A4604461946FFF7F0FF86
:1001A000204610BD10B5202A04DB0146203A9140BC
:1001B000002010BD914020239C1A0346E3401943C0
:1001C000904010BD10B5202A04DB0846203AD040EC
:1001D000002110BD0B46D340D0402024A21A9140EC
:1001E0000843194610BD0000064C0125064E05E0E7
:1001F000E36807CC2B430C3C98471034B442F7D348
:10020000FFF762FF5420000874200008704770B5A3
:100210000024014620314A79022A03D00421C16317
:10022000012418E0026813680E25AB4313600268CE
:1002300013685B085B001360436C1C2213400122AF
:1002400015469D40036C5D604A7100220A71816B06
:10025000002900D08847204670BD0000F8B5002373
:100260000124A2E027469F403A4070D04D68022DFD
:1002700001D0122D14D1DD08AD002D1800952D6A86
:100280005E07AC46F50E0F26AE46AE406546B5435A
:10029000AC460E697546AE4065462E43009D2E6203
:1002A0004D68012D05D0022D03D0112D01D0122D46
:1002B00016D185680326AC465D00AE46AE40654665
:1002C000B543AC46CE687546AE4065462E43866063
:1002D00046680D79BE43ED06ED0F9D403543456000
:1002E00006685F000325BD40AE46AE430D79B446B7
:1002F000AE07B60FBE4065462E430660C66875461B
:10030000AE438D68BD403543C5604D68ED004BD5AB
:10031000294D6E6B26436E639E08284DB6007519F5
:10032000AC46AD689E07360F0F27B740BD43052783
:100330003F07B84201D1002715E0214FB84201D153
:10034000012710E01F4FB84202D102270BE02BE03B
:100350001D4FB84201D1032705E01C4FB84201D11F
:10036000052700E00627B7402F436546AF60184DCC
:100370002E684F689643FF0300D516432E606E68C3
:100380004F689643BF0300D516436E60AE684F6852
:100390009643FF0200D51643AE60EE684F68964361
:1003A000BF0200D51643EE605B1C0A681546DD40AF
:1003B00000D057E7F8BD00000010024000000140E7
:1003C0000004005000080050000C0050001C0050B9
:1003D000000401400069084000D001207047002A55
:1003E00001D0816170478162704700000148006858
:1003F000704700000400002070B502464032537878
:10040000202B1CD11378012B19D001231370242425
:100410005470046825689D432560046825681E03A0
:10042000B5432560046825680D43256000680168B0
:1004300019430160202050700020107070BD022010
:1004400070BD70B5024640325378202B1BD1137813
:10045000012B18D0012414702423537003681D68E5
:10046000A5431D6005682B680F263602B3430902B9
:100470001943296000680168214301602020507001
:100480000020107070BD022070BD000070B5040027
:1004900006D02546403568780026002802D005E0C1
:1004A000012070BD2E70204600F04AF824206870AC
:1004B000206801684908490001600F216068090649
:1004C00088432168086121688A680120C00382434B
:1004D0008A60E1680129A16808D0212292021143B3
:1004E00022689160E168022902D005E00143F7E744
:1004F00001212268C902516021684A680F4B1A43E2
:100500004A602168CA688243CA60616920690843F9
:10051000A169090208432168C860216AE0690843AB
:100520002168086020680168012211430160666447
:10053000202068702663AE70002070BD008000022D
:1005400010B586B0044614216846FFF720FE114915
:10055000206888421BD1104CE16A02200143E1620D
:10056000E16A014003200591800200901220019071
:10057000012002900320039006200490694607485A
:10058000FFF76CFEA06B012189050843A06306B04C
:1005900010BD000000580040001002400004005050
:1005A00002480168491C01607047000004000020F7
:1005B00010B508480024016840221143016020461C
:1005C00000F00AF8002801D0012401E000F01CF836
:1005D000204610BD0020024070B5054609487D2127
:1005E0000024C9000068FFF785FD00F013FE002815
:1005F00001D0012404E000222946501E00F024F816
:10060000204670BD0800002010B50948416B01224A
:1006100011434163816B020411438163002211463F
:10062000042000F011F8042000F004F810BD0000D0
:1006300000100240C106C90E01208840014908602F
:100640007047000000E100E010B501F0AFF810BD08
:10065000F8B504460078544D800672D5524E0027F6
:10066000403EB06BC00004D4B06BA9050843B06332
:1006700001274E480168C90511D40168821511434C
:100680000160FFF7B3FE009005E0FFF7AFFE0099B1
:10069000401A642837D845480068C005F5D5326847
:1006A0000321090560680A400140914208D0810396
:1006B000890F032904D13168890301D50120F8BDD0
:1006C0002A69032109040A4022D0084090421FD021
:1006D000207880061CD528692A6988430121C9042D
:1006E0000A432A612A698A432A612861C0050FD515
:1006F000FFF77CFE009008E0FFF778FE0099411AB2
:100700002B48814201D90320F8BD28698005F3D523
:1007100061688803800F032805D132680005824391
:1007200001400A43326028690322616812041140C3
:1007300008432861002F04D0B16B012000078143DA
:10074000B1632078C00705D0E868A1688008800000
:100750000843E8602078800705D5E8680C218843C5
:10076000E1680843E8602078400706D5E86803217F
:100770008902884321690843E8602078000706D58C
:10078000E86803210903884361690843E860207829
:10079000000606D5E868032189048843A169084357
:1007A000E8600020F8BD00004010024000700040EA
:1007B00088130000F8B50E4605007DD05348006848
:1007C000C007C00FB0420AD250480168490849002A
:1007D000314301600068C007C00FB04271D1287872
:1007E0004B4C800705D5E068F0218843A968084391
:1007F000E0602878C00752D06868022817D0032824
:1008000018D02168012818D08905002959DAE16833
:10081000890889000143E160FFF7E8FD6968074640
:10082000022912D003291CD0012926D033E02168E7
:100830008903EAE721688901E7E74907E5E7FFF768
:10084000D5FDC11B3348814223D8E0680007800FE3
:100850000228F4D123E0FFF7C9FDC11B2D488142D6
:1008600017D8E0680007800F0328F4D117E0FFF7DE
:10087000BDFDC11B274881420BD8E0680007800FEF
:100880000128F4D10BE0FFF7B1FDC11B21488142E3
:1008900001D90320F8BDE0680007800FF3D11B48A1
:1008A0000168C907C90FB1420DD90168490849005B
:1008B00031430160006800E003E0C007C00FB042B0
:1008C00001D00120F8BD2878400706D5E06807214F
:1008D00009028843E9680843E0602878000707D5E3
:1008E000E0680721C90288432969C9000843E0601C
:1008F00000F036F8E168084A0906090F515CC84063
:10090000064908600020FFF767FEF8BD002002409E
:10091000001002408813000030200008080000206A
:10092000044805490068C968044A4905490F515CF3
:10093000C84070470800002000100240492000080D
:10094000044805490068C968044A8904490F515C94
:10095000C8407047080000200010024049200008ED
:1009600010B5184AD1680C20084004280BD008287C
:1009700010D00C2810D050680004410F0120C00393
:10098000491C884010BD1068C00601D50E4810BD36
:100990000E4810BD0E4810BD88020E4B000F185CAB
:1009A0000902D368890F491CDB0301D5084A05E019
:1009B0001268D20601D5044A00E0044A5043FFF70A
:1009C00099FB10BD0010024000093D000024F40016
:1009D00000127A0040200008FEB505007ED0FE4CD3
:1009E000E7680C20E66807400120000406402878EC
:1009F000C00747D0082F05D00C2F0AD101200004D2
:100A0000864206D1206880033CD568680028E5D07E
:100A100038E0012069680004814203D12168014364
:100A2000216011E0052301221B04920499422168F0
:100A300002D111432160F1E7814321602168014027
:100A40000091206890432060686800280DD0FFF76F
:100A5000CDFC009005E0FFF7C9FC0099401A64281E
:100A60007AD820688003F6D50CE0FFF7BFFC009031
:100A700005E0FFF7BBFC0099401A6428F0D8206815
:100A80008003F6D42878800755D50923E868042F19
:100A90000DD00C2F01D1002E09D000283BD02168A9
:100AA000994301432160FFF7A1FC064627E0216836
:100AB000490701D5002891D061681F221202914395
:100AC0002A69120211436160216899430143216040
:100AD000FFF746FFE16809060A0F00E079E1BF4928
:100AE000895CC840BE4908600020FFF775FD0028FA
:100AF00072D120E0FFF77AFC801B0228B0D8206872
:100B00004007F7D560681F21090288432969090257
:100B1000084360600FE02068400840002060FFF755
:100B200065FC064604E0FFF761FC801B022897D8AD
:100B300020684007F7D42878C0065FD5002F0CD076
:100B4000A869002849D02068FF21013108432060AE
:100B5000FFF74CFC06462DE0C0E02068800502D57A
:100B6000A8690028A7D06068072149038843296A3B
:100B7000084360606068297F0002000A0906084394
:100B80006060286A410B0120C003491C8840E1686D
:100B900009060A0F9149895CC84091490860002004
:100BA000FFF71AFD002817D128E0FFF71FFC801B74
:100BB0000228A3D820688005F7D56068072149037B
:100BC0008843296A084360606068297F0002000A40
:100BD00009060843606011E0E1E02168FF20013070
:100BE00081432160FFF702FC064604E0FFF7FEFBAD
:100BF000801B022872D820688005F7D42878794EA7
:100C0000000724D568690028306910D00121084305
:100C10003061FFF7EBFB009005E0FFF7E7FB009981
:100C2000401A02285AD830698007F6D50FE04008EC
:100C300040003061FFF7DAFB009005E0FFF7D6FBDC
:100C40000099401A022849D830698007F6D42878DC
:100C5000400765D500200290A06BC00006D4A06BB1
:100C6000012109070843A063012002905E48016842
:100C7000C90511D40168821511430160FFF7B6FB65
:100C8000009005E0FFF7B2FB0099401A642825D8D0
:100C900055480068C005F5D5FF20AA68013082429A
:100CA00003D131690143316111E001218902002A38
:100CB00007D005231B029A4203D132690A433261ED
:100CC000EFE7326982433261306988433061A86856
:100CD00000280FD0FFF78AFB009007E05EE0FFF7E7
:100CE00085FB0099411A4148814257D830698005F7
:100CF000F5D50DE0FFF77AFB009006E0FFF776FBF5
:100D00000099411A3948814248D830698005F5D4A4
:100D10000298002804D0A06B012109078843A06332
:100D2000686A002864D00C2F3ED0012636060228BF
:100D3000206805D0B0432060FFF758FB05462FE040
:100D4000B0432060FFF752FB074604E0FFF74EFB7D
:100D5000C01B022822D820688001F7D4E96AA86A5B
:100D6000E2680843296BFD231B049A43114308439F
:100D7000E060206830432060FFF738FB054604E060
:100D8000FFF734FB401B022808D820688001F7D504
:100D90002EE0FFF72BFB401B022801D90320FEBDEC
:100DA00020688001F5D423E00128F8D0E068012113
:100DB0000904AA6A014091420BD10F218904EA6A11
:100DC0000140914205D1032189050840296B8842E1
:100DD0000ED00120FEBD00000010024030200008AF
:100DE00008000020401002400070004088130000FE
:100DF0000020EFE7F7B5054604462035287882B095
:100E0000012814D001202870022068702168CA20AF
:100E100048622168532048622068806800264005A7
:100E2000FF27002812DAFFF7E1FA00900AE002201B
:100E300005B0F0BDFFF7DAFA0099411A7D20C00035
:100E4000814215D82068C0684007F3D420688168C3
:100E50000122920291438160FFF7C8FA00900DE0F1
:100E6000FFF7C4FA0099411A7D20C000814205D9DC
:100E700020684762032068702E70D9E72068C06838
:100E80004007EDD520688168C908C90081602068E5
:100E90008168049A11438160216803984861206841
:100EA000816801229202114381602068476201201B
:100EB00068702E700020BBE710B500680B464068D4
:100EC000C021C94301400002000ECC04D870E40EDA
:100ED0005C708C06A40E0904490F9C701970002ADE
:100EE0000AD100F087FCD870587800F083FC587065
:100EF000987800F07FFC9870002010BD30B50B464C
:100F00000168896A5960016809694904490C996056
:100F1000006804680F482146014088024D04800E95
:100F200018706D0E49065D70490E99706102490E88
:100F300040242140D970002A0AD100F05BFC1870CF
:100F4000587800F057FC5870987800F053FC98706F
:100F5000002030BD7F7F7F00F8B5040050D02546CB
:100F600020356878002803D12870204600F052F818
:100F7000022068702168CA204862216853204862B4
:100F8000204600F04BFCFF2604270028206802D0F2
:100F900046626F7034E081681D4A114081602168AB
:100FA00088686268A369104322691A431043886005
:100FB0002168E068086120680169228912041143F0
:100FC00001612068C16880229143C1602068C16CC2
:100FD00089088900C164E169606901432068C26CC5
:100FE0001143C1642068806880060BD4204600F05D
:100FF000F7F8002806D0206846626F70002028703D
:101000000120F8BD20684662012068700020F8BD0C
:10101000BFFF8FFF00680549884205D10448016978
:101020000122920411430161704700000028004032
:1010300040100240F8B505460446203528780B4696
:1010400001280FD00120287002206870002A0BD0E0
:10105000D8789E780004064358780978000249033E
:10106000084317E00220F8BD5878C10603D5EF21E8
:1010700008400A305870D87800F0C4FB060458784D
:1010800000F0C0FB00020643987800F0BBFB06436B
:101090001878400306432168CA204862216853201B
:1010A0004862204600F0BAFB0027002811D1114801
:1010B0000640206846602068C16880229143C16074
:1010C0002068806880060CD4204600F089F800284B
:1010D00007D02168FF204862042068702F7001202B
:1010E000F8BD2168FF204862012068702F70002041
:1010F000F8BD00003FFFFF00F8B506460446203665
:1011000030780D46012822D0012030700220707006
:10111000206800278068002A1BD0400600D4EF70AA
:101120002978A878090408436978EA780902120442
:101130001143084300902168CA2048622168532067
:101140004862204600F06AFB002837D116E00220F2
:10115000F8BD400600D4EF70287800F053FB03047C
:10116000687800F04FFB00020343A87800F04AFBC8
:101170000343E878000403430093DCE71749009831
:101180000840216808602068816801229204914328
:1011900081602969E868084321688A68104388608B
:1011A0002068C16880229143C16020688068800601
:1011B0000CD4204600F014F8002807D02168FF2046
:1011C00048620420707037700120F8BD2168FF204C
:1011D00048620120707037700020F8BD7F7F7F006B
:1011E00070B504460068C168A0229143C160FFF752
:1011F000FDF87D260546F60006E0FFF7F7F8401BF0
:10120000B04201D9032070BD2068C0688006F4D5C3
:10121000002070BD094910B5401E884201D9012047
:1012200010BD074C60610321081F00F0BFFA0020C9
:10123000A06107202061002010BD0000FFFFFF001B
:1012400000E000E0F0B502462032137E012B15D0FD
:10125000012717760223537605686C68AB68702601
:10126000B4430E68496826438024A34319436E6043
:1012700000688160577600201076F0BD0220F0BD36
:1012800070B5040005D025462035687E002802D0C0
:1012900006E0012070BD00202876204600F00AF804
:1012A00002206876211D206800F03EFB0120687650
:1012B000002070BD00680449884204D10348816B56
:1012C000102211438163704700100040001002405B
:1012D00070477047F8B502680446D0691168936892
:1012E00005072D0F5BD0DD07ED0FFF2621360E40E1
:1012F0002E4367D0C60706D0CE0504D50126166258
:10130000E26F3243E267870702220426002F06DAE3
:10131000DF0704D027683A62E76F3743E76747077C
:1013200006D5DB0704D023681E62E36F1343E3672F
:10133000020709D520220A402A4305D02368082243
:101340001A62E36F1343E367E26F002A2FD080062F
:1013500006D5880604D5216E002901D0204688478D
:10136000E06F21688968490601D4000724D520462A
:1013700000F0A6FB20688168490619D581684022E3
:1013800091438160E06E002812D020498163E06EB5
:10139000FEF73DFF00280AD0E06E816B06E085066F
:1013A00010D58D060ED5216E1CE020468847F8BD6D
:1013B0002046FFF78EFFF8BD2046FFF78AFF00208A
:1013C000E067F8BDC50208D55B0206D5012000051F
:1013D00010622046FFF77CFFF8BD030605D50B061B
:1013E00003D5616E0029E0D1F8BD4006FCD5480662
:1013F000FAD51368204640218B4313602021616792
:101400000021616600F0D7F8F8BD0000AD1A0008B1
:1014100010B5040003D0606F002802D007E001205F
:1014200010BD002170200155204600F027F824202F
:10143000606720680168490849000160204600F0A3
:101440004FFB0128ECD0606A002802D0204600F053
:1014500097FA206841680922D202914341602068CE
:1014600081682A229143816020680168012211432A
:101470000160204600F0EAFA10BD000010B586B009
:10148000044614216846FEF782FE1549206888420A
:1014900024D11448416B0122920311434163C16A74
:1014A00001221143C162C06A6946104005900320C1
:1014B000400200900220019000200290032003903F
:1014C0000420049005200007FEF7C8FE0022114604
:1014D0001B20FFF7B9F81B20FFF7ACF806B010BDD2
:1014E0000038014000100240FFB50446406F83B051
:1014F00017460D4620285CD1002D0AD0002F08D0B9
:10150000A168C001814207D12069002804D1E80701
:1015100002D0012007B0F0BD204660300290007C70
:10152000012846D00298012101740020E0672120A3
:101530006067FEF75BFF2646403601903782778270
:101540000120A1680003814202D12069002802D055
:101550002F46002511E000270FE0002280212046C1
:1015600000F0D2FB002815D1002F15D02168387863
:1015700088627F1C708A401E7082708A019B0028DE
:1015800006980090E9D100224021204600F0BCFBE3
:10159000002808D00320BDE728882168C005C00DB9
:1015A0008862AD1CE6E7202060670299002008747D
:1015B000B0E70220AEE77047FEE70000F0B587B065
:1015C00014216846FEF7E3FD1C48C16A0125294342
:1015D000C162C16A29400591C26A02210A43C262FE
:1015E000C06AC1260840052776013F070590002202
:1015F00031463846FEF7F3FE002270211048FEF710
:10160000EEFE1020002400900194694602943846B2
:10161000FEF724FE0294694638460096019503942D
:10162000FEF71CFE70200090029469460195039419
:101630000348FEF713FE07B0F0BD000000100240A3
:101640000004005010B5134811490160124941606F
:10165000002181600161416181610122C161C2603B
:101660000162FEF713FF002801D0FEF7CFFD002135
:101670000848FEF7C1FE002801D0FEF7C7FD002193
:101680000448FEF7DEFE002801D0FEF7BFFD10BDC6
:1016900000580040240000200E09002010B586B03C
:1016A00014216846FEF773FD00241E491E48059468
:1016B00012C07F2101608460C4600461FF21446125
:1016C00041600838FFF748FC002801D0FEF79EFD76
:1016D000684604704470847003940122694612487D
:1016E0000494FFF709FD002801D0FEF78FFD0120CB
:1016F0006946087548758875CC75024605A90A487B
:10170000FFF798FC002801D0FEF780FD002211466B
:101710000548FFF76FFB002801D0FEF777FD06B004
:1017200010BD000000280040700000201CB50024FF
:101730000E4800940C4901940160072184604160C7
:1017400001214461C160FFF79BFD002801D0FEF735
:101750005DFD0094694605480194FFF773FD00287C
:1017600001D0FEF753FD1CBD001000409400002086
:1017700010B50C480A490160E1214902416000218D
:101780008160C16001618161C1610C2201624261BD
:101790004162FFF73DFE002801D0FEF737FD10BD86
:1017A00000380140D0000020704700008307FF226E
:1017B000DB0E9A408907090E994000280BDA0007D2
:1017C000000F0838830808489B001818C369934322
:1017D0000B43C3617047830804489B001B181868BB
:1017E000904308431860704700ED00E000E400E01B
:1017F0007047704701090A2200075143000F401843
:10180000C0B270470022014602E00A39C9B2521C38
:101810000A29FAD21007000E0843704770B5044633
:101820000068C168490613D40021C943C160FEF7AE
:10183000DDFD7D260546F60006E0FEF7D7FD401BE0
:10184000B04201D9032070BD2068C0684006F4D5BD
:10185000002070BD704710B5FEF7A2FE10BD00005D
:1018600030B599B034216846FEF791FC14210DA8DB
:10187000FEF78DFC1C2112A8FEF789FC14480168B4
:101880000322D2029143C214891801600A200090F9
:1018900000240125102009940490039505956846BD
:1018A000FFF79AF80F200D9080200F900E9510945E
:1018B000002111940DA8FEF77DFF212012906804ED
:1018C0001390149412A8FEF7C3FE19B030BD0000A7
:1018D0000070004010480168821511430160C16822
:1018E0000E4A1140C16001680D4A114001608168D3
:1018F0004908490081600168012292049143016016
:10190000C168FD2212049143C160002101610549B3
:10191000C003886070470000001002400C40FF8840
:10192000F6FFF6FE00ED00E070B5026801239B07AC
:10193000114C124D984203D0A04201D0A84203D1CD
:101940007026B2434E683243984203D0A04201D081
:10195000A84204D103231B029A43CB681A43802375
:101960009A430B691A4302608A68C26209688162FD
:101970000121416170BD00000008014000140140D8
:1019800010B5818CC90707D001684A6801235B0440
:101990009A43836A1A434A60818C890707D5016894
:1019A0004A6801231B049A43C36A1A434A60818C24
:1019B000490707D501684A6801239B049A43036BD2
:1019C0001A434A60818C090707D501684A680123D8
:1019D000DB039A43436B1A434A60818CC90607D5DF
:1019E0000268916801231B039943836B194391603B
:1019F000818C890607D501688A6801235B039A43B5
:101A0000C36B1A438A60818C490612D503685A68F1
:101A100001210905046C8A4322435A60026C8A4200
:101A200007D10268516803235B059943436C19434E
:101A30005160818C090607D501684A680123DB04DF
:101A4000806C9A4302434A6010BD0000F8B500263E
:101A50000446C667FEF7CAFC054620680068124FB8
:101A6000000709D501212B46002249052046009791
:101A700000F04AF900280DD12068006840070BD516
:101A800001212B46002289052046009700F03CF9F1
:101A9000002801D00320F8BD20206067A0676034D3
:101AA00026740020F8BD0000FFFFFF0110B5806A1A
:101AB0000022014640314A834A82FFF70AFC10BDEA
:101AC00001680A68FF2321339A430A6001688A6823
:101AD000520852008A602021816700210166704708
:101AE000F8B504462669A268E769324366691020A2
:101AF00000253E432368324378491E68784F3E40B4
:101B000016431E6023685A6803263603B243E6680C
:101B100032435A602368A2698B4201D0266A32435D
:101B20009E680B273F02BE4316439E606D4E23689E
:101B30006D4AB3420CD1D2689207920F06D0012AA7
:101B400038D0022A34D0032A20D11EE001201DE023
:101B5000664EB3420AD1D2680C26324026D0042AFF
:101B600028D0082A24D00C2A10D10EE08B420DD1A7
:101B7000D66803229202164018D001229202B61AA9
:101B800018D0B61A14D0964200D10820564A012621
:101B9000403A574FF6038B4236D100280CD002282A
:101BA0000DD0042812D008281FD11CE00020EDE73A
:101BB0000220EBE70420E9E7FEF7B2FE08E0106838
:101BC000C00601D5384605E04A4803E0FEF7C8FEE6
:101BD000002873D0626851005118814205D8110362
:101BE000814202D303E03046F4E7012566E0010EAE
:101BF00006025008002330185941FEF791FA0321DC
:101C00000902411A3C4A55E0E169B14232D1030070
:101C100000F0C4F809070A0D06250606062B060083
:101C2000E3E7FEF77DFE1CE0FEF78AFE19E0106890
:101C30006168C00602D54808304A01E0304A4808C9
:101C40008018FEF757FA80B201462E4A10399142A9
:101C5000CBD8511C01400007400F08432CE0FEF791
:101C60007FFE616840004A08EAE76168012248088F
:101C70001204E5E7030000F091F809070A0D0626B3
:101C80000606062C0600B0E7FEF74AFE1DE0FEF74A
:101C900057FE1AE010686168C00602D54808C019EE
:101CA00002E014484A081018FEF724FA80B20146F0
:101CB000144A1039914298D82168C86000202066E3
:101CC00060662846F8BDFEF74BFE61684A0880183A
:101CD000EAE7616848088019E6E70000004800402C
:101CE000F369FFEF0038014040100240004400401B
:101CF00000093D000024F400FFFC0F0000127A00F0
:101D00000048E801EFFF0000FFB581B017460E461E
:101D100004460A9D09E0681C07D0FEF767FB04999A
:101D2000401AA8420CD8002D0AD02068C16930465C
:101D3000884318D00020B842EDD0002005B0F0BD97
:101D400020680168FF22A132914301602068816808
:101D500049084900816020206067A0670020603446
:101D600020740320EAE70120E5E7000010B50248EF
:101D7000FFF7B0FA10BD0000D00000200FB410B57E
:101D800003A9044B044A029800F024F810BC08BCD4
:101D900004B01847251F00080C00002030B474461A
:101DA000641E2578641CAB4200D21D46635D5B0057
:101DB000E31830BC184702E008C8121F08C1002A07
:101DC000FAD170477047002001E001C1121F002ABC
:101DD000FBD17047FFB58DB00446002506E02528ED
:101DE0000AD0109A0F999047641C6D1C2078002827
:101DF000F5D1284611B0F0BD00270121484A0097CF
:101E000000E00743641C23780846203B98401042BA
:101E1000F7D120782E2817D1042007436078641C5E
:101E20002A280CD10E98641C02C800910E900BE079
:101E300000990A22514330394018641C00902078E0
:101E4000014630390929F3D920780028D1D06428F7
:101E500008D0692806D075281ED0109A0F9990478F
:101E60006D1C5BE00A200E99019001C90E910028BB
:101E700002DA40422D2102E0390504D52B216A46C1
:101E80001172012103E0F90704D02021F7E70BAE1E
:101E90000B910DE00021FAE70A200E99019001C98B
:101EA0000E91F7E70199FEF725F93031761E317072
:101EB0000028F7D103A8801B20300190780701D5B6
:101EC000009801E0012000900199884201DD401A4C
:101ED00000E000200027009006E002A8109AC05DF4
:101EE0000F9990476D1C7F1C0B988742F5DB04E02F
:101EF000109A30200F9990476D1C0099481E009051
:101F00000029F5DC05E03078109A761C0F9990478F
:101F10006D1C0199481E01900029F4DC641C65E7E2
:101F20000928010001B5044B012269460348FFF767
:101F3000DBFA009808BD0000FFFF0000D000002081
:101F4000FEF736FBFFF78CFC0024FFF737FBFFF7AB
:101F50000FFCFFF7EBFBFFF775FBFFF79FFB002282
:101F600023492448FEF7CAFF002223492148FEF7EF
:101F7000A3FF1F48052746783F0700221C491D483C
:101F8000FEF7BCFF00221C491A48FEF795FF1848CF
:101F9000102145783846FEF71DFA002806D1102199
:101FA0003846FEF717FA012800D1641CB542E4D088
:101FB0002E460A2C02DA214610A011E0642C02DA27
:101FC000214611A00CE07D20C000844202DA2146A7
:101FD00010A005E07D200001844204DA21460FA014
:101FE000FFF7CCFE02E00FA0FFF7C8FE0024C4E715
:101FF000100000207000002000000020463030302B
:102000002564440D0A0000004630302564440D0A62
:102010000000000046302564440D0A004625644453
:102020000D0A00004639393939440D0A0000000014
:102030000000000000000000010203040607080978
:10204000030406080C1018203000000000010203F1
:1020500004000000742000080000002010000000B0
:10206000B61D000884200008100000204005000074
:10207000C61D000800000000000000000000200055
:04208000000000005C
:04000005080000C12E
:00000001FF
